******************************************************************************
             TMS320C2000 Linker PC v22.6.0                     
******************************************************************************
>> Linked Fri Apr 28 00:00:11 2023

OUTPUT FILE NAME:   <28388D_TEMP_CPU1.out>
ENTRY POINT SYMBOL: "code_start"  address: 00080000


MEMORY CONFIGURATION

         name            origin    length      used     unused   attr    fill
----------------------  --------  ---------  --------  --------  ----  --------
  BOOT_RSVD             00000002   000001af  00000000  000001af  RWIX
  RAMM0                 000001b1   0000024f  00000000  0000024f  RWIX
  RAMM1                 00000400   000003f8  00000200  000001f8  RWIX
  RAMLS0                00008000   00000800  00000043  000007bd  RWIX
  RAMLS1                00008800   00000800  00000000  00000800  RWIX
  RAMLS2                00009000   00000800  00000000  00000800  RWIX
  RAMLS3                00009800   00000800  00000000  00000800  RWIX
  RAMLS4                0000a000   00000800  00000000  00000800  RWIX
  RAMLS5                0000a800   00000800  00000010  000007f0  RWIX
  RAMLS6                0000b000   00000800  00000000  00000800  RWIX
  RAMLS7                0000b800   00000800  00000000  00000800  RWIX
  RAMD0                 0000c000   00000800  00000000  00000800  RWIX
  RAMD1                 0000c800   00000800  00000000  00000800  RWIX
  RAMGS0                0000d000   00001000  00000000  00001000  RWIX
  RAMGS1                0000e000   00001000  00000000  00001000  RWIX
  RAMGS2                0000f000   00001000  00000000  00001000  RWIX
  RAMGS3                00010000   00001000  00000000  00001000  RWIX
  RAMGS4                00011000   00001000  00000000  00001000  RWIX
  RAMGS5                00012000   00001000  00000000  00001000  RWIX
  RAMGS6                00013000   00001000  00000000  00001000  RWIX
  RAMGS7                00014000   00001000  00000000  00001000  RWIX
  RAMGS8                00015000   00001000  00000000  00001000  RWIX
  RAMGS9                00016000   00001000  00000000  00001000  RWIX
  RAMGS10               00017000   00001000  00000000  00001000  RWIX
  RAMGS11               00018000   00001000  00000000  00001000  RWIX
  RAMGS12               00019000   00001000  00000000  00001000  RWIX
  RAMGS13               0001a000   00001000  00000000  00001000  RWIX
  RAMGS14               0001b000   00001000  00000000  00001000  RWIX
  RAMGS15               0001c000   00000ff8  00000000  00000ff8  RWIX
  CMTOCPURAM            00038000   00000800  00000088  00000778  RWIX
  CPUTOCMRAM            00039000   00000800  00000088  00000778  RWIX
  CPU1TOCPU2RAM         0003a000   00000800  00000088  00000778  RWIX
  CPU2TOCPU1RAM         0003b000   00000800  00000088  00000778  RWIX
  CANA_MSG_RAM          00049000   00000800  00000000  00000800  RWIX
  CANB_MSG_RAM          0004b000   00000800  00000000  00000800  RWIX
  BEGIN                 00080000   00000002  00000002  00000000  RWIX
  FLASH0                00080002   00001ffe  00000000  00001ffe  RWIX
  FLASH1                00082000   00002000  00000af8  00001508  RWIX
  FLASH2                00084000   00002000  00000000  00002000  RWIX
  FLASH3                00086000   00002000  00000043  00001fbd  RWIX
  FLASH4                00088000   00008000  00000014  00007fec  RWIX
  FLASH5                00090000   00008000  00000088  00007f78  RWIX
  FLASH6                00098000   00008000  00000000  00008000  RWIX
  FLASH7                000a0000   00008000  00000000  00008000  RWIX
  FLASH8                000a8000   00008000  00000000  00008000  RWIX
  FLASH9                000b0000   00008000  00000000  00008000  RWIX
  FLASH10               000b8000   00002000  00000000  00002000  RWIX
  FLASH11               000ba000   00002000  00000000  00002000  RWIX
  FLASH12               000bc000   00002000  00000000  00002000  RWIX
  FLASH13               000be000   00001ff0  00000000  00001ff0  RWIX
  RESET                 003fffc0   00000002  00000000  00000002  RWIX


SECTION ALLOCATION MAP

 output                                  attributes/
section   page    origin      length       input sections
--------  ----  ----------  ----------   ----------------
codestart 
*          0    00080000    00000002     
                  00080000    00000002     f2838x_codestartbranch.obj (codestart)

.cinit     0    00088000    00000014     
                  00088000    0000000a     (.cinit..data.load) [load image, compression = lzss]
                  0008800a    00000004     (__TI_handler_table)
                  0008800e    00000002     --HOLE-- [fill = 0]
                  00088010    00000004     (__TI_cinit_table)

.reset     0    003fffc0    00000000     DSECT

.stack     0    00000400    00000200     UNINITIALIZED
                  00000400    00000200     --HOLE--

.init_array 
*          0    00082000    00000000     UNINITIALIZED

.data      0    0000a800    00000010     UNINITIALIZED
                  0000a800    00000006     cpu1_isr.obj (.data)
                  0000a806    00000006     rts2800_fpu64_eabi.lib : exit.c.obj (.data)
                  0000a80c    00000002                            : _lock.c.obj (.data:_lock)
                  0000a80e    00000002                            : _lock.c.obj (.data:_unlock)

MSGRAM_CM_TO_CPU 
*          0    00038000    00000088     UNINITIALIZED
                  00038000    00000088     ipc.obj (MSGRAM_CM_TO_CPU)

MSGRAM_CPU_TO_CM 
*          0    00039000    00000088     UNINITIALIZED
                  00039000    00000088     ipc.obj (MSGRAM_CPU_TO_CM)

.const     0    00090000    00000088     
                  00090000    00000088     ipc.obj (.const:IPC_Instance)

MSGRAM_CPU1_TO_CPU2 
*          0    0003a000    00000088     UNINITIALIZED
                  0003a000    00000088     ipc.obj (MSGRAM_CPU1_TO_CPU2)

MSGRAM_CPU2_TO_CPU1 
*          0    0003b000    00000088     UNINITIALIZED
                  0003b000    00000088     ipc.obj (MSGRAM_CPU2_TO_CPU1)

.TI.ramfunc 
*          0    00086000    00000043     RUN ADDR = 00008000
                  00086000    0000003f     flash.obj (.TI.ramfunc:Flash_initModule)
                  0008603f    00000004     sysctl.obj (.TI.ramfunc)

.text      0    00082000    00000af8     
                  00082000    00000167     device.obj (.text:Device_enableAllPeripherals)
                  00082167    00000109     sysctl.obj (.text:SysCtl_setClock)
                  00082270    00000104     sysctl.obj (.text:SysCtl_isPLLValid)
                  00082374    000000e4     sysctl.obj (.text:SysCtl_setAuxClock)
                  00082458    000000d3     dcc.obj (.text:DCC_verifyClockFrequency)
                  0008252b    00000088     rts2800_fpu64_eabi.lib : fs_div28.asm.obj (.text)
                  000825b3    0000006d     cpu1_board.obj (.text:EPWM_init)
                  00082620    00000048     device.obj (.text:Device_init)
                  00082668    00000041     interrupt.obj (.text:Interrupt_initModule)
                  000826a9    0000003f     gpio.obj (.text:GPIO_setPadConfig)
                  000826e8    00000039     sysctl.obj (.text:SysCtl_selectOscSourceAuxPLL)
                  00082721    00000036     cpu1_board.obj (.text:GPIO_init)
                  00082757    00000036     interrupt.obj (.text:Interrupt_enable)
                  0008278d    00000030     gpio.obj (.text:GPIO_setPinConfig)
                  000827bd    0000002f     cpu1_board.obj (.text:PinMux_init)
                  000827ec    0000002e     rts2800_fpu64_eabi.lib : copy_decompress_lzss.c.obj (.text:decompress:lzss)
                  0008281a    0000002b                            : autoinit.c.obj (.text:__TI_auto_init_nobinit_nopinit)
                  00082845    00000029                            : exit.c.obj (.text)
                  0008286e    00000028     sysctl.obj (.text:SysCtl_selectXTAL)
                  00082896    00000026     sysctl.obj (.text:SysCtl_selectOscSource)
                  000828bc    00000023     sysctl.obj (.text:SysCtl_pollX1Counter)
                  000828df    00000022     gpio.obj (.text:GPIO_setControllerCore)
                  00082901    00000022     gpio.obj (.text:GPIO_setQualificationMode)
                  00082923    00000020     gpio.obj (.text:GPIO_setDirectionMode)
                  00082943    0000001f     cpu1_isr.obj (.text:INT_mEPWM5_ISR)
                  00082962    0000001e     device.obj (.text:Device_initGPIO)
                  00082980    0000001d     rts2800_fpu64_eabi.lib : memcpy.c.obj (.text)
                  0008299d    0000001c     device.obj (.text:Device_verifyXTAL)
                  000829b9    0000001c     sysctl.obj (.text:SysCtl_selectXTALSingleEnded)
                  000829d5    0000001b     device.obj (.text:Device_enableUnbondedGPIOPullups)
                  000829f0    00000019     device.obj (.text:SysCtl_enablePeripheral)
                  00082a09    00000019     rts2800_fpu64_eabi.lib : boot28.asm.obj (.text)
                  00082a22    00000017     sysctl.obj (.text:SysCtl_controlCMReset)
                  00082a39    00000015     device.obj (.text:Device_bootCM)
                  00082a4e    00000015     device.obj (.text:Device_bootCPU2)
                  00082a63    00000015     interrupt.obj (.text:Interrupt_initVectorTable)
                  00082a78    00000015     sysctl.obj (.text:SysCtl_controlCPU2Reset)
                  00082a8d    00000015     cpu1_main.obj (.text:main)
                  00082aa2    00000011     cpu1_board.obj (.text:Board_init)
                  00082ab3    0000000c     cpu1_board.obj (.text:INTERRUPT_init)
                  00082abf    0000000c     rts2800_fpu64_eabi.lib : args_main.c.obj (.text)
                  00082acb    00000009     epwm.obj (.text:EPWM_setEmulationMode)
                  00082ad4    00000009     rts2800_fpu64_eabi.lib : _lock.c.obj (.text)
                  00082add    00000008                            : copy_decompress_none.c.obj (.text:decompress:none)
                  00082ae5    00000008     f2838x_codestartbranch.obj (.text)
                  00082aed    00000004     interrupt.obj (.text:Interrupt_defaultHandler)
                  00082af1    00000002     interrupt.obj (.text:Interrupt_illegalOperationHandler)
                  00082af3    00000002     interrupt.obj (.text:Interrupt_nmiHandler)
                  00082af5    00000002     rts2800_fpu64_eabi.lib : pre_init.c.obj (.text)
                  00082af7    00000001                            : startup.c.obj (.text)

MODULE SUMMARY

       Module                       code   ro data   rw data
       ------                       ----   -------   -------
    .\
       cpu1_board.obj               239    0         0      
       cpu1_isr.obj                 31     0         6      
       cpu1_main.obj                21     0         0      
    +--+----------------------------+------+---------+---------+
       Total:                       291    0         6      
                                                            
    .\device\
       device.obj                   583    0         0      
       f2838x_codestartbranch.obj   10     0         0      
    +--+----------------------------+------+---------+---------+
       Total:                       593    0         0      
                                                            
    .\device\driverlib\
       sysctl.obj                   1003   0         0      
       ipc.obj                      0      136       544    
       dcc.obj                      211    0         0      
       gpio.obj                     211    0         0      
       interrupt.obj                148    0         0      
       flash.obj                    126    0         0      
       epwm.obj                     9      0         0      
    +--+----------------------------+------+---------+---------+
       Total:                       1708   136       544    
                                                            
    E:\soft ware\ti\ccs1200\ccs\tools\compiler\ti-cgt-c2000_22.6.0.LTS\lib\rts2800_fpu64_eabi.lib
       fs_div28.asm.obj             136    0         0      
       exit.c.obj                   41     0         6      
       copy_decompress_lzss.c.obj   46     0         0      
       autoinit.c.obj               43     0         0      
       memcpy.c.obj                 29     0         0      
       boot28.asm.obj               25     0         0      
       _lock.c.obj                  9      0         4      
       args_main.c.obj              12     0         0      
       copy_decompress_none.c.obj   8      0         0      
       pre_init.c.obj               2      0         0      
       startup.c.obj                1      0         0      
    +--+----------------------------+------+---------+---------+
       Total:                       352    0         10     
                                                            
       Stack:                       0      0         512    
       Linker Generated:            0      18        0      
    +--+----------------------------+------+---------+---------+
       Grand Total:                 2944   154       1072   


LINKER GENERATED COPY TABLES

__TI_cinit_table @ 00088010 records: 1, size/record: 4, table size: 4
	.data: load addr=00088000, load size=0000000a bytes, run addr=0000a800, run size=00000010 bytes, compression=lzss


LINKER GENERATED HANDLER TABLE

__TI_handler_table @ 0008800a records: 2, size/record: 2, table size: 4
	index: 0, handler: __TI_decompress_lzss
	index: 1, handler: __TI_decompress_none


GLOBAL DATA SYMBOLS: SORTED BY DATA PAGE

address     data page           name
--------    ----------------    ----
00000400      10 (00000400)     __stack

0000a800     2a0 (0000a800)     startTime
0000a801     2a0 (0000a800)     endTime
0000a802     2a0 (0000a800)     count
0000a804     2a0 (0000a800)     deltTime
0000a806     2a0 (0000a800)     __TI_enable_exit_profile_output
0000a808     2a0 (0000a800)     __TI_cleanup_ptr
0000a80a     2a0 (0000a800)     __TI_dtors_ptr
0000a80c     2a0 (0000a800)     _lock
0000a80e     2a0 (0000a800)     _unlock

00038000     e00 (00038000)     IPC_CPU_To_CM_GetBuffer

00039000     e40 (00039000)     IPC_CPU_To_CM_PutBuffer

0003a000     e80 (0003a000)     IPC_CPU1_To_CPU2_PutBuffer

0003b000     ec0 (0003b000)     IPC_CPU1_To_CPU2_GetBuffer

00090000    2400 (00090000)     IPC_Instance


GLOBAL SYMBOLS: SORTED ALPHABETICALLY BY Name 

page  address   name                            
----  -------   ----                            
0     00082aa2  Board_init                      
0     00082845  C$$EXIT                         
0     00082458  DCC_verifyClockFrequency        
0     00082a39  Device_bootCM                   
0     00082a4e  Device_bootCPU2                 
0     00082000  Device_enableAllPeripherals     
0     000829d5  Device_enableUnbondedGPIOPullups
0     00082620  Device_init                     
0     00082962  Device_initGPIO                 
0     0008299d  Device_verifyXTAL               
0     000825b3  EPWM_init                       
0     00082acb  EPWM_setEmulationMode           
0     00008000  Flash_initModule                
0     00082721  GPIO_init                       
0     000828df  GPIO_setControllerCore          
0     00082923  GPIO_setDirectionMode           
0     000826a9  GPIO_setPadConfig               
0     0008278d  GPIO_setPinConfig               
0     00082901  GPIO_setQualificationMode       
0     00082ab3  INTERRUPT_init                  
0     00082943  INT_mEPWM5_ISR                  
0     0003b000  IPC_CPU1_To_CPU2_GetBuffer      
0     0003a000  IPC_CPU1_To_CPU2_PutBuffer      
0     00038000  IPC_CPU_To_CM_GetBuffer         
0     00039000  IPC_CPU_To_CM_PutBuffer         
0     00090000  IPC_Instance                    
0     00082757  Interrupt_enable                
0     00082668  Interrupt_initModule            
0     00082a63  Interrupt_initVectorTable       
0     000827bd  PinMux_init                     
0     00086043  RamfuncsLoadEnd                 
abs   00000043  RamfuncsLoadSize                
0     00086000  RamfuncsLoadStart               
0     00008043  RamfuncsRunEnd                  
abs   00000043  RamfuncsRunSize                 
0     00008000  RamfuncsRunStart                
0     00082a22  SysCtl_controlCMReset           
0     00082a78  SysCtl_controlCPU2Reset         
0     0000803f  SysCtl_delay                    
0     00082270  SysCtl_isPLLValid               
0     00082896  SysCtl_selectOscSource          
0     000826e8  SysCtl_selectOscSourceAuxPLL    
0     0008286e  SysCtl_selectXTAL               
0     000829b9  SysCtl_selectXTALSingleEnded    
0     00082374  SysCtl_setAuxClock              
0     00082167  SysCtl_setClock                 
0     00088010  __TI_CINIT_Base                 
0     00088014  __TI_CINIT_Limit                
0     00088014  __TI_CINIT_Warm                 
0     0008800a  __TI_Handler_Table_Base         
0     0008800e  __TI_Handler_Table_Limit        
0     00000600  __TI_STACK_END                  
abs   00000200  __TI_STACK_SIZE                 
0     0008281a  __TI_auto_init_nobinit_nopinit  
0     0000a808  __TI_cleanup_ptr                
0     000827ec  __TI_decompress_lzss            
0     00082add  __TI_decompress_none            
0     0000a80a  __TI_dtors_ptr                  
0     0000a806  __TI_enable_exit_profile_output 
abs   ffffffff  __TI_pprof_out_hndl             
abs   ffffffff  __TI_prof_data_size             
abs   ffffffff  __TI_prof_data_start            
0     0008252b  __c28xabi_divf                  
n/a   UNDEFED   __c_args__                      
0     00000400  __stack                         
0     00082abf  _args_main                      
0     00082a09  _c_int00                        
0     0000a80c  _lock                           
0     00082adc  _nop                            
0     00082ad8  _register_lock                  
0     00082ad4  _register_unlock                
0     00082af7  _system_post_cinit              
0     00082af5  _system_pre_init                
0     0000a80e  _unlock                         
0     00082845  abort                           
0     00080000  code_start                      
0     0000a802  count                           
0     0000a804  deltTime                        
0     0000a801  endTime                         
0     00082847  exit                            
0     00082a8d  main                            
0     00082980  memcpy                          
0     0000a800  startTime                       


GLOBAL SYMBOLS: SORTED BY Symbol Address 

page  address   name                            
----  -------   ----                            
0     00000400  __stack                         
0     00000600  __TI_STACK_END                  
0     00008000  Flash_initModule                
0     00008000  RamfuncsRunStart                
0     0000803f  SysCtl_delay                    
0     00008043  RamfuncsRunEnd                  
0     0000a800  startTime                       
0     0000a801  endTime                         
0     0000a802  count                           
0     0000a804  deltTime                        
0     0000a806  __TI_enable_exit_profile_output 
0     0000a808  __TI_cleanup_ptr                
0     0000a80a  __TI_dtors_ptr                  
0     0000a80c  _lock                           
0     0000a80e  _unlock                         
0     00038000  IPC_CPU_To_CM_GetBuffer         
0     00039000  IPC_CPU_To_CM_PutBuffer         
0     0003a000  IPC_CPU1_To_CPU2_PutBuffer      
0     0003b000  IPC_CPU1_To_CPU2_GetBuffer      
0     00080000  code_start                      
0     00082000  Device_enableAllPeripherals     
0     00082167  SysCtl_setClock                 
0     00082270  SysCtl_isPLLValid               
0     00082374  SysCtl_setAuxClock              
0     00082458  DCC_verifyClockFrequency        
0     0008252b  __c28xabi_divf                  
0     000825b3  EPWM_init                       
0     00082620  Device_init                     
0     00082668  Interrupt_initModule            
0     000826a9  GPIO_setPadConfig               
0     000826e8  SysCtl_selectOscSourceAuxPLL    
0     00082721  GPIO_init                       
0     00082757  Interrupt_enable                
0     0008278d  GPIO_setPinConfig               
0     000827bd  PinMux_init                     
0     000827ec  __TI_decompress_lzss            
0     0008281a  __TI_auto_init_nobinit_nopinit  
0     00082845  C$$EXIT                         
0     00082845  abort                           
0     00082847  exit                            
0     0008286e  SysCtl_selectXTAL               
0     00082896  SysCtl_selectOscSource          
0     000828df  GPIO_setControllerCore          
0     00082901  GPIO_setQualificationMode       
0     00082923  GPIO_setDirectionMode           
0     00082943  INT_mEPWM5_ISR                  
0     00082962  Device_initGPIO                 
0     00082980  memcpy                          
0     0008299d  Device_verifyXTAL               
0     000829b9  SysCtl_selectXTALSingleEnded    
0     000829d5  Device_enableUnbondedGPIOPullups
0     00082a09  _c_int00                        
0     00082a22  SysCtl_controlCMReset           
0     00082a39  Device_bootCM                   
0     00082a4e  Device_bootCPU2                 
0     00082a63  Interrupt_initVectorTable       
0     00082a78  SysCtl_controlCPU2Reset         
0     00082a8d  main                            
0     00082aa2  Board_init                      
0     00082ab3  INTERRUPT_init                  
0     00082abf  _args_main                      
0     00082acb  EPWM_setEmulationMode           
0     00082ad4  _register_unlock                
0     00082ad8  _register_lock                  
0     00082adc  _nop                            
0     00082add  __TI_decompress_none            
0     00082af5  _system_pre_init                
0     00082af7  _system_post_cinit              
0     00086000  RamfuncsLoadStart               
0     00086043  RamfuncsLoadEnd                 
0     0008800a  __TI_Handler_Table_Base         
0     0008800e  __TI_Handler_Table_Limit        
0     00088010  __TI_CINIT_Base                 
0     00088014  __TI_CINIT_Limit                
0     00088014  __TI_CINIT_Warm                 
0     00090000  IPC_Instance                    
abs   00000043  RamfuncsLoadSize                
abs   00000043  RamfuncsRunSize                 
abs   00000200  __TI_STACK_SIZE                 
abs   ffffffff  __TI_pprof_out_hndl             
abs   ffffffff  __TI_prof_data_size             
abs   ffffffff  __TI_prof_data_start            
n/a   UNDEFED   __c_args__                      

[83 symbols]
